:020000040000FA
:0408000061EF09F0AB
:1008100003B26EEF05F0F2B48CEF05F09EB094EFEA
:1008200005F09EB29CEF05F0F2A81AEF04F0F2B2C8
:100830001CEF04F010EF09F0CD90F2929EA026EF8D
:1008400004F00101533F26EF04F0542BB2C1B6F17E
:10085000B3C1B7F1B4C1B8F1B5C1B9F1AEC1B2F12C
:10086000AFC1B3F1B0C1B4F1B1C1B5F1AAC1AEF13C
:10087000ABC1AFF1ACC1B0F1ADC1B1F1A6C1AAF14C
:10088000A7C1ABF1A8C1ACF1A9C1ADF1A2C1A6F15C
:10089000A3C1A7F1A4C1A8F1A5C1A9F19EC1A2F16C
:1008A0009FC1A3F1A0C1A4F1A1C1A5F19AC19EF17C
:1008B0009BC19FF19CC1A0F19DC1A1F1CECF9AF146
:1008C000CFCF9BF153C19CF154C19DF1CF6ACE6A49
:1008D0000101536B546B9E90CD800FBC0F8E0FBAED
:1008E00075EF04F00F8A10EF09F013880F8C0FBE1C
:1008F000B2EF04F09AC19EF19BC19FF19CC1A0F19F
:100900009DC1A1F19EC1A2F19FC1A3F1A0C1A4F11B
:10091000A1C1A5F1A2C1A6F1A3C1A7F1A4C1A8F1EB
:10092000A5C1A9F1A6C1AAF1A7C1ABF1A8C1ACF1BB
:10093000A9C1ADF1AAC1AEF1ABC1AFF1ACC1B0F18B
:10094000ADC1B1F1AEC1B2F1AFC1B3F1B0C1B4F15B
:10095000B1C1B5F1B2C1B6F1B3C1B7F1B4C1B8F12B
:10096000B5C1B9F101015E6B5F6B606B616B9A5150
:100970005E279B515F239C5160239D5161239E51B3
:100980005E279F515F23A0516023A1516123A25193
:100990005E27A3515F23A4516023A5516123A65173
:1009A0005E27A7515F23A8516023A9516123AA5153
:1009B0005E27AB515F23AC516023AD516123AE5133
:1009C0005E27AF515F23B0516023B1516123B25113
:1009D0005E27B3515F23B4516023B5516123B651F3
:1009E0005E27B7515F23B8516023B9516123D89076
:1009F0000101613360335F335E33D89001016133AD
:100A000060335F335E33D8900101613360335F330D
:100A10005E3300C10CF101C10DF102C10EF103C141
:100A20000FF104C110F105C111F106C112F107C1A6
:100A300013F108C114F109C115F10AC116F10BC176
:100A400017F134C135F111B831EF05F00101620E33
:100A5000046F010E056F000E066F000E076F3AEF70
:100A600005F00101A70E046F020E056F000E066F60
:100A7000000E076F5EC100F15FC101F160C102F1BC
:100A800061C103F1D1EC1FF003BF04D019BE02D045
:100A900019A0108C11A052EF05F010BA52EF05F01A
:100AA0000F80108A0CC100F10DC101F10EC102F1DD
:100AB0000FC103F110C104F111C105F112C106F11A
:100AC00013C107F114C108F115C109F116C10AF1EA
:100AD00017C10BF135C134F110EF09F00392ABB23D
:100AE000AB98AB88030103EE00F080517F0BE92641
:100AF00004C0EFFF802B8151805D700BD8A48B82E6
:100B000000008051815D700BD8A48B9281518019B7
:100B1000D8B4079010EF09F0F2940101453F10EFAF
:100B200009F0462B10EF09F09E900101533F10EFA2
:100B300009F0542B10EF09F09E9213A0C6EF05F0B8
:100B400001015E6B5F6B606B616B626B636B646B0F
:100B5000656B666B676B686B696B536B546BCF6AC5
:100B6000CE6A0F9A0F9C0F9E0101476B486B496B31
:100B70004A6B4B6B4C6B4D6B4E6B4F6B506B516BB1
:100B8000526B456B466BD76AD66A139011B83AEF31
:100B900007F08BB4D3EF05F010ACD3EF05F08B84E6
:100BA000109CD4EF05F08B94C3CF55F1C4CF56F110
:100BB000C28207B443EF06F047C14BF148C14CF184
:100BC00049C14DF14AC14EF15EC162F15FC163F1AD
:100BD00060C164F161C165F113A8F1EF05F0138CF8
:100BE00013989AC1BAF19BC1BBF19CC1BCF19DC1E4
:100BF000BDF19EC1BEF19FC1BFF1A0C1C0F1A1C1B5
:100C0000C1F1A2C1C2F1A3C1C3F1A4C1C4F1A5C184
:100C1000C5F1A6C1C6F1A7C1C7F1A8C1C8F1A9C154
:100C2000C9F1AAC1CAF1ABC1CBF1ACC1CCF1ADC124
:100C3000CDF1AEC1CEF1AFC1CFF1B0C1D0F1B1C1F4
:100C4000D1F1B2C1D2F1B3C1D3F1B4C1D4F1B5C1C4
:100C5000D5F1B6C1D6F1B7C1D7F1B8C1D8F1B9C194
:100C6000D9F1010155515B2756515C23E86A5D2398
:100C70000E2E43EF06F05CC157F15DC158F15B6B7E
:100C80005C6B5D6B078E0201002F10EF09F03C0ECC
:100C9000006F1A50E00BE00AE866128818BE02D016
:100CA00018B4108E00C10CF101C10DF102C10EF19A
:100CB00003C10FF104C110F105C111F106C112F118
:100CC00007C113F108C114F109C115F10AC116F1E8
:100CD0000BC117F134C135F101018E6777EF06F0D2
:100CE0008F6777EF06F0906777EF06F091677BEFFD
:100CF00006F0ABEF06F092C100F193C101F194C18F
:100D000002F195C103F10101010E046F000E056FA0
:100D1000000E066F000E076FD1EC1FF000C192F1BC
:100D200001C193F102C194F103C195F10067A0EFF5
:100D300006F00167A0EF06F00267A0EF06F0036778
:100D4000ABEF06F08EC192F18FC193F190C194F197
:100D500091C195F10F80D57ED5BE6ED0D6CF47F12B
:100D6000D7CF48F145C149F1E86AE8CF4AF1138A83
:100D700019BE02D019A0108C109047C100F148C1D3
:100D800001F149C102F14AC103F101010A0E046FE8
:100D9000000E056F000E066F000E076FD1EC1FF0FE
:100DA00003AF1080010154A7E2EF06F00F9A0F9CE9
:100DB0000F9E0101000E5E6F600E5F6F3D0E606F53
:100DC000080E616F010147BFF2EF06F04867F2EFCE
:100DD00006F04967F2EF06F04A67F2EF06F0F28894
:100DE00017EF07F0F2985E6B5F6B606B616B9A6B4D
:100DF0009B6B9C6B9D6B9E6B9F6BA06BA16BA26BA7
:100E0000A36BA46BA56BA66BA76BA86BA96BAA6B56
:100E1000AB6BAC6BAD6BAE6BAF6BB06BB16BB26B06
:100E2000B36BB46BB56BB66BB76BB86BB96BD76A9A
:100E3000D66A0101456B466B0CC100F10DC101F191
:100E40000EC102F10FC103F110C104F111C105F18E
:100E500012C106F113C107F114C108F115C109F15E
:100E600016C10AF117C10BF135C134F110EF09F0C9
:100E700010EF09F00201002F94EF08F0D59ED6CFB5
:100E800047F1D7CF48F145C149F1E86AE8CF4AF1C7
:100E9000138AD76AD66A0101456B466BD58E1A5004
:100EA000E00BE00AE866128818BE02D018B4108E73
:100EB00017AE1C8C00C10CF101C10DF102C10EF185
:100EC00003C10FF104C110F105C111F106C112F106
:100ED00007C113F108C114F109C115F10AC116F1D6
:100EE0000BC117F134C135F10FA0109A11B884EF7E
:100EF00007F00101620E046F010E056F000E066F10
:100F0000000E076F8DEF07F00101A70E046F020EB0
:100F1000056F000E066F000E076F47C100F148C154
:100F200001F149C102F14AC103F1D1EC1FF003BF45
:100F3000A0EF07F019BE02D019A0108C11B00F80DD
:100F40000CC100F10DC101F10EC102F10FC103F19D
:100F500010C104F111C105F112C106F113C107F16D
:100F600014C108F115C109F116C10AF117C10BF13D
:100F700035C134F102013C0E006F00C10CF101C11A
:100F80000DF102C10EF103C10FF104C110F105C151
:100F900011F106C112F107C113F108C114F109C121
:100FA00015F10AC116F10BC117F134C135F1010178
:100FB0008E67E2EF07F08F67E2EF07F09067E2EFEE
:100FC00007F09167E6EF07F016EF08F092C100F125
:100FD00093C101F194C102F195C103F10101010E28
:100FE000046F000E056F000E066F000E076FD1EC48
:100FF0001FF000C192F101C193F102C194F103C14C
:1010000095F100670BEF08F001670BEF08F002673E
:101010000BEF08F0036716EF08F08EC192F18FC155
:1010200093F190C194F191C195F10F80109047C157
:1010300000F148C101F149C102F14AC103F10101C6
:101040000A0E046F000E056F000E066F000E076F8C
:10105000D1EC1FF003AF1080010154A73CEF08F062
:101060000F9A0F9C0F9E0101000E5E6F600E5F6F66
:101070003D0E606F080E616F47C100F148C101F17C
:1010800049C102F14AC103F10101140E046F050EBA
:10109000056F000E066F000E076FD1EC1FF003AF57
:1010A00055EF08F0F2887AEF08F0F2985E6B5F6B0C
:1010B000606B616B9A6B9B6B9C6B9D6B9E6B9F6B6C
:1010C000A06BA16BA26BA36BA46BA56BA66BA76BAC
:1010D000A86BA96BAA6BAB6BAC6BAD6BAE6BAF6B5C
:1010E000B06BB16BB26BB36BB46BB56BB66BB76B0C
:1010F000B86BB96B0CC100F10DC101F10EC102F169
:101100000FC103F110C104F111C105F112C106F1C3
:1011100013C107F114C108F115C109F116C10AF193
:1011200017C10BF135C134F18BB49EEF08F010AC50
:101130009EEF08F08B84109C9FEF08F08B94C3CF38
:1011400055F1C4CF56F1C28207B40EEF09F047C182
:101150004BF148C14CF149C14DF14AC14EF15EC15C
:1011600062F15FC163F160C164F161C165F113A80F
:10117000BCEF08F0138C13989AC1BAF19BC1BBF174
:101180009CC1BCF19DC1BDF19EC1BEF19FC1BFF12B
:10119000A0C1C0F1A1C1C1F1A2C1C2F1A3C1C3F1FB
:1011A000A4C1C4F1A5C1C5F1A6C1C6F1A7C1C7F1CB
:1011B000A8C1C8F1A9C1C9F1AAC1CAF1ABC1CBF19B
:1011C000ACC1CCF1ADC1CDF1AEC1CEF1AFC1CFF16B
:1011D000B0C1D0F1B1C1D1F1B2C1D2F1B3C1D3F13B
:1011E000B4C1D4F1B5C1D5F1B6C1D6F1B7C1D7F10B
:1011F000B8C1D8F1B9C1D9F1010155515B27565198
:101200005C23E86A5D230E2E0EEF09F05CC157F1F6
:101210005DC158F15B6B5C6B5D6B078E10EF09F085
:1012200002C0E0FF005001C0D8FF1000A6B216EFC8
:1012300009F00CC0A9FF0BC0A8FFA69EA69CA6841F
:10124000F29E550EA76EAA0EA76EA682F28EA694E7
:10125000A6B228EF09F00C2A1200A96EA69EA69C41
:10126000A680A8500C2A120004012C0E826F3CECC0
:101270000BF0CCEC20F00C502DEC09F0E8CF00F195
:101280000C502DEC09F0E8CF01F101AF4DEF09F062
:101290000101FF0E026FFF0E036F6FEC20F0296754
:1012A00059EF09F00401200E826F3CEC0BF05EEF69
:1012B00009F004012D0E826F3CEC0BF079EC1EF06E
:1012C0001200306A076A0F6A106A116A126A136A9A
:1012D0000F010E0EC16E860EC06E030EC26E0F01A0
:1012E000896A110E926E080E8A6EF10E936E8B6AE9
:1012F000800E946EF18E81848286FC0E2DEC09F0B6
:10130000E8CF0BF00BA011800BA211820BA411846B
:101310000BA81188C90E2DEC09F0E8CF17F0CA0E02
:101320002DEC09F0E8CF18F0CB0E2DEC09F0E8CF4A
:1013300019F0CC0E2DEC09F0E8CF1AF0CD0E2DEC03
:1013400009F0E8CF2FF01C6A1D6A0E6A01015B6B81
:101350005C6B5D6B576B586BF29A0101476B486B86
:10136000496B4A6B4B6B4C6B4D6B4E6B4F6B506BC1
:10137000516B526B456B466BD76AD66A0F01280ECC
:10138000D56EF28A9D90B00ECD6E01015E6B5F6BE3
:10139000606B616B626B636B646B656B666B676BD9
:1013A000686B696B536B546BCF6ACE6A0F9A0F9C54
:1013B0000F9E9D80760ECA6E9D8202013C0E006FCC
:1013C000CC6A160E2DEC09F0E8CF00F1170E2DECCB
:1013D00009F0E8CF01F1180E2DEC09F0E8CF02F189
:1013E000190E2DEC09F0E8CF03F1010103AF13EF63
:1013F0000AF0CCEC20F0160E0C6E00C10BF016ECCF
:1014000009F0170E0C6E01C10BF016EC09F0180E66
:101410000C6E02C10BF016EC09F0190E0C6E03C134
:101420000BF016EC09F000C18EF101C18FF102C181
:1014300090F103C191F100C192F101C193F102C198
:1014400094F103C195F11A0E2DEC09F0E8CF00F1EB
:101450001B0E2DEC09F0E8CF01F11C0E2DEC09F06C
:10146000E8CF02F11D0E2DEC09F0E8CF03F10101E8
:1014700003AF69EF0AF0CCEC20F01A0E0C6E00C13D
:101480000BF016EC09F01B0E0C6E01C10BF016EC04
:1014900009F01C0E0C6E02C10BF016EC09F01D0ECB
:1014A0000C6E03C10BF016EC09F01A0E2DEC09F0CE
:1014B000E8CF00F11B0E2DEC09F0E8CF01F11C0E76
:1014C0002DEC09F0E8CF02F11D0E2DEC09F0E8CF6C
:1014D00003F100C196F101C197F102C198F103C176
:1014E00099F1240EAC6E900EAB6E240EAC6E080E0D
:1014F000B86E000EB06E1F0EAF6E0401806B816B74
:101500000F01900EAB6E0F019D8A0301806B816B02
:10151000C26B8B9207900001F28EF28C07B027EF1E
:101520001DF00FB038EF16F010BE38EF16F012B8FD
:1015300038EF16F00301805181197F0BD8B427EFE3
:101540001DF013EE00F081517F0BE126812BE7CFD8
:10155000E8FFE00BD8B427EF1DF023EE82F0C25174
:101560003F0BD926E7CFDFFFC22BDF50780AD8A484
:1015700027EF1DF0078092C100F193C101F194C1E2
:1015800002F195C103F10101040E046F000E056F15
:10159000000E066F000E076FD1EC1FF000AFDAEF00
:1015A0000AF00101030E926F000E936F000E946F0C
:1015B000000E956F03018251720AD8B414EF16F031
:1015C0008251520AD8B414EF16F08251750AD8B479
:1015D00014EF16F08251630AD8B4E1EF19F082518A
:1015E000690AD8B4BEEF12F082517A0AD8B4D1EFAA
:1015F00013F08251490AD8B40FEF12F08251500A09
:10160000D8B42DEF11F08251700AD8B470EF11F0F8
:101610008251540AD8B49BEF11F08251740AD8B4A5
:10162000E1EF11F08251410AD8B452EF0CF082512F
:101630004B0AD8B450EF0BF082516D0AD8B485EF45
:1016400010F082514D0AD8B49EEF10F08251730A07
:10165000D8B444EF15F08251530AD8B4A9EF15F06D
:101660008251660AD8B470EF12F08251590AD8B488
:10167000D6EF0FF018EF1AF0040114EE00F08051CD
:101680007F0BE12682C4E7FF802B120004010D0EC0
:10169000826F3CEC0BF00A0E826F3CEC0BF01200F8
:1016A00004014B0E826F3CEC0BF004012C0E826F98
:1016B0003CEC0BF081B802D02FB630D0030183513F
:1016C000430AD8B495EF0BF003018351630AD8B4F1
:1016D00097EF0BF003018351520AD8B499EF0BF046
:1016E00003018351720AD8B49BEF0BF003018351BD
:1016F000470AD8B49DEF0BF003018351670AD8B4B1
:101700009FEF0BF003018351540AD8B4A1EF0BF003
:1017100003018351740AD8B410EF0CF00301835114
:10172000550AD8B4A3EF0BF082D02F807AD02F9037
:1017300078D02F8276D02F9274D02F8472D02F94AD
:1017400070D02F866ED084C330F185C331F186C34B
:1017500032F187C333F10101296B1AEC21F091ECCE
:1017600020F000C104F101C105F102C106F103C17D
:1017700007F10DEC21F0200EF86EF76AF66A090009
:10178000F5CF2CF10900F5CF2DF10900F5CF2EF1A1
:101790000900F5CF2FF10900F5CF30F10900F5CFA1
:1017A00031F10900F5CF32F10900F5CF33F1010134
:1017B000296B1AEC21F091EC20F0D1EC1FF00067BE
:1017C000E9EF0BF00167E9EF0BF00267E9EF0BF0CF
:1017D000036701D025D004014E0E826F3CEC0BF064
:1017E00004016F0E826F3CEC0BF004014D0E826F12
:1017F0003CEC0BF00401610E826F3CEC0BF0040139
:10180000740E826F3CEC0BF00401630E826F3CECB3
:101810000BF00401680E826F3CEC0BF016EF1AF02F
:101820002F96CD0E0C6E2FC00BF016EC09F0CD0EDE
:101830002DEC09F0E8CF2FF02FB006D00401630E95
:10184000826F3CEC0BF005D00401430E826F3CEC40
:101850000BF02FB206D00401720E826F3CEC0BF03D
:1018600005D00401520E826F3CEC0BF02FB406D071
:101870000401670E826F3CEC0BF005D00401470EAB
:10188000826F3CEC0BF02FB606D00401740E826F11
:101890003CEC0BF005D00401540E826F3CEC0BF0D5
:1018A00016EF1AF00401410E826F3CEC0BF00301BD
:1018B0008351310AD8B4F6EF0EF003018351320A96
:1018C000D8B426EF0EF003018351330AD8B4AFEF3A
:1018D0000DF003018351340AD8B49FEF0CF00301DB
:1018E0008351350AD8B47CEF0CF004013F0E826FAF
:1018F0003CEC0BF016EF1AF004012C0E826F3CEC5E
:101900000BF003018451300AD8B48FEF0CF00301BF
:101910008451310AD8B497EF0CF0E8EF0DF08B90BA
:101920000401300E826F3CEC0BF09DEF0CF08B80CD
:101930000401310E826F3CEC0BF016EF1AF0CC0E66
:101940002DEC09F0E8CF0BF004012C0E826F3CEC7B
:101950000BF003018451310AD8B4C3EF0CF003013A
:101960008451300AD8B4C5EF0CF0030184514D0AFC
:10197000D8B4CFEF0CF003018451540AD8B4D6EF99
:101980000CF0EDEF0CF08A8401D08A940BAE04D0F9
:101990000BAC02D00BBA21D0E00E0B1218D01F0EE8
:1019A0000B168539E844E00B0B1211D0E00E0B1634
:1019B0000DEC21F085C332F186C333F10101296BAF
:1019C0001AEC21F091EC20F000511F0B0B12CC0E01
:1019D0000C6E0BC00BF016EC09F00401340E826F94
:1019E0003CEC0BF004012C0E826F3CEC0BF0CC0EA7
:1019F0002DEC09F0E8CF1AF08AB406D00401300EBD
:101A0000826F3CEC0BF005D00401310E826F3CEC90
:101A10000BF004012C0E826F3CEC0BF01A38E840FE
:101A2000070BE8CF82F40401300E82273CEC0BF068
:101A300004012C0E826F3CEC0BF0CCEC20F01A5021
:101A40001F0BE8CF00F16FEC20F032C182F40401EB
:101A5000300E82273CEC0BF033C182F40401300ECF
:101A600082273CEC0BF004012C0E826F3CEC0BF057
:101A7000CCEC20F02DC000F100AF0BD0FF0E016FB9
:101A8000FF0E026FFF0E036F04012D0E826F3CEC00
:101A90000BF06FEC20F031C182F40401300E82278C
:101AA0003CEC0BF032C182F40401300E82273CEC96
:101AB0000BF033C182F40401300E82273CEC0BF0B2
:101AC00004012C0E826F3CEC0BF0CCEC20F02CC00F
:101AD00000F16FEC20F031C182F40401300E822756
:101AE0003CEC0BF032C182F40401300E82273CEC56
:101AF0000BF033C182F40401300E82273CEC0BF072
:101B000004012C0E826F3CEC0BF0CCEC20F02EC0CC
:101B100000F100AF0BD0FF0E016FFF0E026FFF0E42
:101B2000036F04012D0E826F3CEC0BF06FEC20F084
:101B300031C182F40401300E82273CEC0BF032C13B
:101B400082F40401300E82273CEC0BF033C182F4A6
:101B50000401300E82273CEC0BF016EF1AF0CB0E8E
:101B60002DEC09F0E8CF0BF004012C0E826F3CEC59
:101B70000BF003018451450AD8B4D3EF0DF00301F3
:101B80008451440AD8B4D6EF0DF003018451300AD1
:101B9000D8B4D9EF0DF003018451310AD8B4DDEF88
:101BA0000DF0E8EF0DF00B9EE2EF0DF00B8EE2EF83
:101BB0000DF0FC0E0B16E2EF0DF0FC0E0B160B8079
:101BC000E2EF0DF0CB0E0C6E0BC00BF016EC09F033
:101BD0000401330E826F3CEC0BF004012C0E826F7B
:101BE0003CEC0BF0CB0E2DEC09F0E8CF19F019BE50
:101BF00001EF0EF00401450E826F3CEC0BF006EF96
:101C00000EF00401440E826F3CEC0BF004012C0E2C
:101C1000826F3CEC0BF00401300E826F3CEC0BF059
:101C200004012C0E826F3CEC0BF019B01FEF0EF08C
:101C30000401300E826F3CEC0BF024EF0EF0040137
:101C4000310E826F3CEC0BF016EF1AF0CA0E2DEC41
:101C500009F0E8CF0BF004012C0E826F3CEC0BF086
:101C600003018451450AD8B462EF0EF00301845198
:101C7000440AD8B465EF0EF0030184514D0AD8B47C
:101C80006EEF0EF003018451410AD8B468EF0EF0F4
:101C900003018451460AD8B46BEF0EF0030184515E
:101CA000560AD8B476EF0EF003018451500AD8B426
:101CB00081EF0EF003018451520AD8B484EF0EF084
:101CC0008DEF0EF00B9E87EF0EF00B8E87EF0EF070
:101CD0000B9C87EF0EF00B8C87EF0EF0FC0E0B16B3
:101CE00085C3E8FF030B0B1287EF0EF0C70E0B1630
:101CF00085C3E8FF070BE846E846E8460B1287EF86
:101D00000EF00B8487EF0EF00B9487EF0EF0CA0EE7
:101D10000C6E0BC00BF016EC09F0CA0E2DEC09F09E
:101D2000E8CF18F00401320E826F3CEC0BF0040196
:101D30002C0E826F3CEC0BF018BEA6EF0EF00401E7
:101D4000450E826F3CEC0BF0ABEF0EF00401440E3D
:101D5000826F3CEC0BF004012C0E826F3CEC0BF01C
:101D600018C0E8FF030BE8CF82F40401300E82278D
:101D70003CEC0BF004012C0E826F3CEC0BF018BC19
:101D8000C9EF0EF00401410E826F3CEC0BF0CEEF78
:101D90000EF00401460E826F3CEC0BF004012C0E99
:101DA000826F3CEC0BF018C0E8FF380BE842E842C9
:101DB000E842E8CF82F40401300E82273CEC0BF0BD
:101DC00004012C0E826F3CEC0BF018B4EFEF0EF018
:101DD0000401520E826F3CEC0BF0F4EF0EF00401A4
:101DE000500E826F3CEC0BF016EF1AF0C90E2DEC82
:101DF00009F0E8CF0BF004012C0E826F3CEC0BF0E5
:101E000003018451450AD8B414EF0FF00301845143
:101E1000440AD8B417EF0FF0030184514D0AD8B427
:101E20001AEF0FF028EF0FF00B9E22EF0FF00B8E42
:101E300022EF0FF0F80E0B1685C3E8FF070B0B120D
:101E400022EF0FF0C90E0C6E0BC00BF016EC09F070
:101E50000401310E826F3CEC0BF004012C0E826FFA
:101E60003CEC0BF0C90E2DEC09F0E8CF17F017BED3
:101E700006D00401450E826F3CEC0BF005D0040146
:101E8000440E826F3CEC0BF004012C0E826F3CEC94
:101E90000BF017C0E8FF070BE8CF82F40401300E07
:101EA00082273CEC0BF004012C0E826F3CEC0BF013
:101EB0000780CCEC20F028C0E8FF003B0043004343
:101EC000030B6FEC20F033C182F40401300E822743
:101ED0003CEC0BF004012C0E826F3CEC0BF0CCECD4
:101EE00020F028C001F1019F019D29C000F10101EE
:101EF0006FEC20F02FC182F40401300E82273CECFD
:101F00000BF030C182F40401300E82273CEC0BF060
:101F100031C182F40401300E82273CEC0BF032C157
:101F200082F40401300E82273CEC0BF033C182F4C2
:101F30000401300E82273CEC0BF004012C0E826F62
:101F40003CEC0BF0CCEC20F02AC001F12BC000F1EE
:101F5000D89001330033D8900133003301016FEC86
:101F600020F02FC182F40401300E82273CEC0BF0EC
:101F700030C182F40401300E82273CEC0BF031C1F9
:101F800082F40401300E82273CEC0BF032C182F463
:101F90000401300E82273CEC0BF033C182F40401C3
:101FA000300E82273CEC0BF016EF1AF0FC0E2DECF5
:101FB00009F0E8CF0BF003018351520AD8B40DEFBA
:101FC00010F003018351720AD8B410EF10F003012E
:101FD0008351500AD8B413EF10F003018351700AF3
:101FE000D8B416EF10F003018351550AD8B419EF95
:101FF00010F003018351750AD8B41CEF10F00301EF
:102000008351430AD8B425EF10F003018351630ACA
:10201000D8B428EF10F031EF10F00B902BEF10F048
:102020000B802BEF10F00B922BEF10F00B822BEFAD
:1020300010F00B942BEF10F00B842BEF10F00B969D
:102040002BEF10F00B862BEF10F00B982BEF10F00E
:102050000B882BEF10F0FC0E0C6E0BC00BF016EC87
:1020600009F00401590E826F3CEC0BF011901192B3
:1020700011941198FC0E2DEC09F0E8CF0BF00BA099
:1020800011800BA211820BA411840BA8118811A03E
:1020900051EF10F00401520E826F3CEC0BF056EF42
:1020A00010F00401720E826F3CEC0BF011A860EF8F
:1020B00010F00401430E826F3CEC0BF065EF10F062
:1020C0000401630E826F3CEC0BF011A26FEF10F075
:1020D0000401500E826F3CEC0BF074EF10F0040121
:1020E000700E826F3CEC0BF011A47EEF10F0040137
:1020F000550E826F3CEC0BF083EF10F00401750E6F
:10210000826F3CEC0BF016EF1AF004016D0E826F3B
:102110003CEC0BF003018351300AD8B4DDEF10F032
:1021200003018351310AD8B4F0EF10F00301835159
:10213000320AD8B403EF11F018EF1AF004014D0E73
:10214000826F3CEC0BF00DEC21F084C331F185C3C0
:1021500032F186C333F10101296B1AEC21F091ECC5
:1021600020F003018351300AD8B4C5EF10F0030109
:102170008351310AD8B4CDEF10F003018351320AF4
:10218000D8B4D5EF10F018EF1AF0FD0E0C6E00C1A8
:102190000BF016EC09F0DDEF10F0FE0E0C6E00C136
:1021A0000BF016EC09F0F0EF10F0FF0E0C6E00C112
:1021B0000BF016EC09F003EF11F00401300E826F02
:1021C0003CEC0BF004012C0E826F3CEC0BF0CCECE1
:1021D00020F0FD0E2DEC09F0E8CF00F114EF11F026
:1021E0000401310E826F3CEC0BF004012C0E826F67
:1021F0003CEC0BF0CCEC20F0FE0E2DEC09F0E8CF1F
:1022000000F114EF11F00401320E826F3CEC0BF080
:10221000CCEC20F004012C0E826F3CEC0BF0FF0E96
:102220002DEC09F0E8CF00F16FEC20F031C182F421
:102230000401300E82273CEC0BF032C182F4040121
:10224000300E82273CEC0BF033C182F40401300ED7
:1022500082273CEC0BF016EF1AF083C32AF184C3FB
:102260002BF185C32CF186C32DF187C32EF188C3D2
:102270002FF189C330F18AC331F18BC332F18CC3A2
:1022800033F101011AEC21F091EC20F0160E0C6EE6
:1022900000C10BF016EC09F0170E0C6E01C10BF02B
:1022A00016EC09F0180E0C6E02C10BF016EC09F0DA
:1022B000190E0C6E03C10BF016EC09F000C18EF183
:1022C00001C18FF102C190F103C191F100C192F1FE
:1022D00001C193F102C194F103C195F10FEF12F026
:1022E00083C32AF184C32BF185C32CF186C32DF15E
:1022F00087C32EF188C32FF189C330F18AC331F12E
:102300008BC332F18CC333F101011AEC21F091EC53
:1023100020F000C18EF101C18FF102C190F103C123
:1023200091F100C192F101C193F102C194F103C195
:1023300095F10FEF12F083C32AF184C32BF185C30B
:102340002CF186C32DF187C32EF188C32FF189C3E9
:1023500030F18AC331F18CC332F18DC333F1010105
:102360001AEC21F091EC20F00101000E046F000E38
:10237000056F010E066F000E076FE2EC1FF01A0EDC
:102380000C6E00C10BF016EC09F01B0E0C6E01C1B7
:102390000BF016EC09F01C0E0C6E02C10BF016ECE3
:1023A00009F01D0E0C6E03C10BF016EC09F000C114
:1023B00096F101C197F102C198F103C199F10FEFB4
:1023C00012F083C32AF184C32BF185C32CF186C399
:1023D0002DF187C32EF188C32FF189C330F18AC351
:1023E00031F18CC332F18DC333F101011AEC21F0CC
:1023F00091EC20F00101000E046F000E056F010E3C
:10240000066F000E076FE2EC1FF000C196F101C1EC
:1024100097F102C198F103C199F10FEF12F0160E76
:102420002DEC09F0E8CF00F1170E2DEC09F0E8CF04
:1024300001F1180E2DEC09F0E8CF02F1190E2DEC88
:1024400009F0E8CF03F16FEC20F032EC1EF004014C
:10245000730E826F3CEC0BF004012C0E826F3CEC8F
:102460000BF08EC100F18FC101F190C102F191C159
:1024700003F16FEC20F032EC1EF00401730E826F5A
:102480003CEC0BF004012C0E826F3CEC0BF01A0EAE
:102490002DEC09F0E8CF00F11B0E2DEC09F0E8CF90
:1024A00001F11C0E2DEC09F0E8CF02F11D0E2DEC10
:1024B00009F0E8CF03F133EC1AF004012C0E826F1F
:1024C0003CEC0BF096C100F197C101F198C102F10B
:1024D00099C103F133EC1AF046EC0BF018EF1AF047
:1024E0000401660E826F3CEC0BF003018351780A05
:1024F000D8B491EF12F0030183B102D0829601D0DB
:10250000828683B302D0819401D0818484B102D0C9
:10251000829A01D0828A84B302D0829801D08288C4
:10252000138095EC12F016EF1AF004012C0E826F56
:102530003CEC0BF0300E82B602D0E89001D0E8807F
:1025400081B402D0E89201D0E882E8CF82F43CEC7A
:102550000BF004012C0E826F3CEC0BF0300E82BAB3
:1025600002D0E89001D0E88082B802D0E89201D091
:10257000E882E8CF82F43CEC0BF012000401690E13
:10258000826F3CEC0BF004012C0E826F3CEC0BF0E4
:102590000101040E006F000E016F000E026F000EAD
:1025A000036F6FEC20F02CC182F40401300E8227FF
:1025B0003CEC0BF02DC182F40401300E82273CEC80
:1025C0000BF02EC182F40401300E82273CEC0BF09C
:1025D0002FC182F40401300E82273CEC0BF030C195
:1025E00082F40401300E82273CEC0BF031C182F4FE
:1025F0000401300E82273CEC0BF032C182F404015E
:10260000300E82273CEC0BF033C182F40401300E13
:1026100082273CEC0BF004012C0E826F3CEC0BF09B
:102620000101040E006F000E016F000E026F000E1C
:10263000036F6FEC20F02CC182F40401300E82276E
:102640003CEC0BF02DC182F40401300E82273CECEF
:102650000BF02EC182F40401300E82273CEC0BF00B
:102660002FC182F40401300E82273CEC0BF030C104
:1026700082F40401300E82273CEC0BF031C182F46D
:102680000401300E82273CEC0BF032C182F40401CD
:10269000300E82273CEC0BF033C182F40401300E83
:1026A00082273CEC0BF004012C0E826F3CEC0BF00B
:1026B00001013A0E006F000E016F000E026F000E56
:1026C000036F6FEC20F02CC182F40401300E8227DE
:1026D0003CEC0BF02DC182F40401300E82273CEC5F
:1026E0000BF02EC182F40401300E82273CEC0BF07B
:1026F0002FC182F40401300E82273CEC0BF030C174
:1027000082F40401300E82273CEC0BF031C182F4DC
:102710000401300E82273CEC0BF032C182F404013C
:10272000300E82273CEC0BF033C182F40401300EF2
:1027300082273CEC0BF004012C0E826F3CEC0BF07A
:10274000200EF86EF76AF66A04010900F5CF82F4EC
:102750003CEC0BF00900F5CF82F43CEC0BF00900E7
:10276000F5CF82F43CEC0BF00900F5CF82F43CECA1
:102770000BF00900F5CF82F43CEC0BF00900F5CF2B
:1027800082F43CEC0BF00900F5CF82F43CEC0BF04A
:102790000900F5CF82F43CEC0BF046EC0BF018EF9F
:1027A0001AF08351630AD8A416EF1AF08451610A13
:1027B000D8A416EF1AF085516C0AD8A416EF1AF0B7
:1027C0008651410A3FE08651440A1BE08651420A85
:1027D000D8B435EF14F08651350AD8B4A2EF1BF007
:1027E0008651360AD8B4F7EF1BF08651370AD8B4B1
:1027F00060EF1CF08651380AD8B4BEEF1CF016EF1B
:102800001AF00798079A04017A0E826F3CEC0BF0DD
:102810000401780E826F3CEC0BF00401640E826FB1
:102820003CEC0BF00401550E826F3CEC0BF01EEFFC
:1028300014F004014C0E826F3CEC0BF046EC0BF0F4
:1028400018EF1AF00788079A04017A0E826F3CECA1
:102850000BF00401410E826F3CEC0BF00401610EA1
:10286000826F3CEC0BF012EF14F00798078A04011A
:102870007A0E826F3CEC0BF00401420E826F3CEC4E
:102880000BF00401610E826F3CEC0BF012EF14F0C0
:102890000101666753EF14F0676753EF14F0686740
:1028A00053EF14F0696715D04F675EEF14F050676F
:1028B0005EEF14F051675EEF14F052670AD0010129
:1028C000000E006F000E016F000E026F000E036F0E
:1028D000120011B80AD00101620E046F010E056FDB
:1028E000000E066F000E076F09D00101A70E046FDE
:1028F000020E056F000E066F000E076F66C100F135
:1029000067C101F168C102F169C103F1D1EC1FF0A7
:1029100003BFFBEF14F0119A119C0101000E046F2C
:10292000A80E056F550E066F020E076F66C100F107
:1029300067C101F168C102F169C103F166C18AF1A1
:1029400067C18BF168C18CF169C18DF1D1EC1FF0C9
:1029500003BF0BD00101000E8A6FA80E8B6F550EBE
:102960008C6F020E8D6F118A119C0E0E2DEC09F0EA
:10297000E8CF18F10F0E2DEC09F0E8CF19F1100E89
:102980002DEC09F0E8CF1AF1110E2DEC09F0E8CF8B
:102990001BF11AEC1FF08AC104F18BC105F18CC147
:1029A00006F18DC107F1D1EC1FF00782DEEC1EF0BD
:1029B0001AEC1FF00792DEEC1EF08AC100F18BC109
:1029C00001F18CC102F18DC103F10792DEEC1EF022
:1029D000CC0E046FE00E056F870E066F050E076FB5
:1029E000D1EC1FF000C118F101C119F102C11AF1B7
:1029F00003C11BF140D013AA00EF15F0138E139AF8
:102A0000119C119A0101800E006F1A0E016F060EC3
:102A1000026F000E036F4FC104F150C105F151C1A7
:102A200006F152C107F1D1EC1FF003AF05D0CCEC99
:102A300020F0118C119A12000E0E2DEC09F0E8CF47
:102A400018F10F0E2DEC09F0E8CF19F1100E2DEC56
:102A500009F0E8CF1AF1110E2DEC09F0E8CF1BF1C7
:102A60004FC100F150C101F151C102F152C103F156
:102A70000782DEEC1EF018C100F119C101F11AC184
:102A800002F11BC103F112000401730E826F3CECD2
:102A90000BF004012C0E826F3CEC0BF0078462C13A
:102AA00066F163C167F164C168F165C169F14BC149
:102AB0004FF14CC150F14DC151F14EC152F157C1CE
:102AC00059F158C15AF107946AEC15F046EC0BF035
:102AD00018EF1AF066C100F167C101F168C102F197
:102AE00069C103F101016FEC20F032EC1EF004012A
:102AF000630E826F3CEC0BF004012C0E826F3CECF9
:102B00000BF04FC100F150C101F151C102F152C1AE
:102B100003F101016FEC20F032EC1EF00401660EAF
:102B2000826F3CEC0BF004012C0E826F3CEC0BF03E
:102B3000CCEC20F059C100F15AC101F101016FEC58
:102B400020F032EC1EF00401740E826F3CEC0BF0AE
:102B5000120010820401530E826F3CEC0BF0040152
:102B60002C0E826F3CEC0BF083C32AF184C32BF153
:102B700085C32CF186C32DF187C32EF188C32FF1B5
:102B800089C330F18AC331F18BC332F18CC333F185
:102B900001011AEC21F091EC20F000C166F101C1B5
:102BA00067F102C168F103C169F18EC32AF18FC3D5
:102BB0002BF190C32CF191C32DF192C32EF193C34D
:102BC0002FF194C330F195C331F196C332F197C31D
:102BD00033F101011AEC21F091EC20F000C14FF12A
:102BE00001C150F102C151F103C152F10DEC21F0CC
:102BF00099C32FF19AC330F19BC331F19CC332F1D9
:102C00009DC333F101011AEC21F091EC20F000C1D9
:102C100059F101C15AF16AEC15F004012C0E826FD2
:102C20003CEC0BF024EF16F0118E19A002D019AE77
:102C3000108C18BE02D018A4108E03018251520AC3
:102C400002E10F8201D00F928251750A02E11084D5
:102C500001D010948251550A02E1108601D01096DD
:102C60008351310A03E11382138402D01392139427
:102C700011A003D011A401D01084078410B2A2EFD8
:102C800016F010A486EF16F0BAC166F1BBC167F169
:102C9000BCC168F1BDC169F1BEC16AF1BFC16BF1D0
:102CA000C0C16CF1C1C16DF1C2C16EF1C3C16FF1A0
:102CB000C4C170F1C5C171F1C6C172F1C7C173F170
:102CC000C8C174F1C9C175F1CAC176F1CBC177F140
:102CD000CCC178F1CDC179F1CEC17AF1CFC17BF110
:102CE000D0C17CF1D1C17DF1D2C17EF1D3C17FF1E0
:102CF000D4C180F1D5C181F1D6C182F1D7C183F1B0
:102D0000D8C184F1D9C185F18EEF16F062C166F1A8
:102D100063C167F164C168F165C169F1BAC186F147
:102D2000BBC187F1BCC188F1BDC189F14BC14FF175
:102D30004CC150F14DC151F14EC152F157C159F141
:102D400058C15AF107940FA0C4EF16F0010196671D
:102D5000B1EF16F09767B1EF16F09867B1EF16F084
:102D60009967B5EF16F0C4EF16F048EC14F096C171
:102D700004F197C105F198C106F199C107F1D1ECB1
:102D80001FF003BFDCEF19F048EC14F00101000E56
:102D9000046F000E056F010E066F000E076F02EC48
:102DA00020F011A02AD011A228D06FEC20F02967C2
:102DB00001D005D004012D0E826F3CEC0BF030C128
:102DC00082F40401300E82273CEC0BF031C182F416
:102DD0000401300E82273CEC0BF032C182F4040176
:102DE000300E82273CEC0BF033C182F40401300E2C
:102DF00082273CEC0BF046EC0BF012A8C5D01298E1
:102E00001AC01BF01B3A1B42070E1B1600011B5079
:102E1000000AD8B490EF17F000011B50010AD8B493
:102E20001CEF17F000011B50020AD8B41AEF17F07C
:102E3000C2EF17F0C2EF17F0CCEC20F02AC001F17E
:102E40002BC000F1D89001330033D8900133003308
:102E50000101630E046F000E056F000E066F000E79
:102E6000076F02EC20F0280E046F000E056F000EB5
:102E7000066F000E076FD1EC1FF000C12DF0CCECF7
:102E800020F028C001F1019F019D29C000F101013E
:102E9000A40E046F000E056F000E066F000E076F84
:102EA00002EC20F000C12CF000C104F101C105F1D9
:102EB00002C106F103C107F1640E006F000E016F3D
:102EC000000E026F000E036FD1EC1FF0050E046FB1
:102ED000000E056F000E066F000E076F02EC20F06B
:102EE00000C104F101C105F102C106F103C107F1FE
:102EF000CCEC20F02DC000F1D1EC1FF000C12EF081
:102F00002EC0E8FF050F2D5C03E78A84C2EF17F09F
:102F10002EC0E8FF0A0F2D5C01E68A94C2EF17F07D
:102F200000C124F101C125F102C126F103C127F13D
:102F3000CCEC20F0D2EC20F01A501F0BE8CF00F1BF
:102F40000101640E046F000E056F000E066F000E87
:102F5000076FE2EC1FF024C104F125C105F126C181
:102F600006F127C107F1D1EC1FF003BF02D08A940C
:102F700001D08A8424C100F125C101F126C102F1EA
:102F800027C103F118EF1AF000C124F101C125F1A6
:102F900002C126F103C127F110AE4DD0109E00C131
:102FA00008F101C109F102C10AF103C10BF16FEC93
:102FB00020F030C1DAF131C1DBF132C1DCF133C1D3
:102FC000DDF108C100F109C101F10AC102F10BC133
:102FD00003F101016C0E046F070E056F000E066F02
:102FE000000E076FD1EC1FF003BF04D00101550E96
:102FF000DE6F1CD008C100F109C101F10AC102F164
:103000000BC103F10101A40E046F060E056F000E43
:10301000066F000E076FD1EC1FF003BF04D0010153
:103020007F0EDE6F03D00101FF0EDE6F1C8E11AE2E
:10303000DCEF19F0119E24C100F125C101F126C178
:1030400002F127C103F111A005D011A203D00FB0E6
:10305000DCEF19F010A434EF18F00401750E826F44
:103060003CEC0BF039EF18F00401720E826F3CEC6F
:103070000BF004012C0E826F3CEC0BF06FEC20F097
:10308000296748EF18F00401200E826F4BEF18F00B
:1030900004012D0E826F3CEC0BF030C182F4040170
:1030A000300E82273CEC0BF031C182F40401300E6B
:1030B00082273CEC0BF004012E0E826F3CEC0BF0EF
:1030C00032C182F40401300E82273CEC0BF033C194
:1030D00082F40401300E82273CEC0BF004016D0EEB
:1030E000826F3CEC0BF004012C0E826F3CEC0BF079
:1030F0004FC100F150C101F151C102F152C103F1C0
:1031000001016FEC20F032EC1EF00401480E826FDA
:103110003CEC0BF004017A0E826F3CEC0BF00401E6
:103120002C0E826F3CEC0BF066C100F167C101F11F
:1031300068C102F169C103F101016FEC20F032ECCA
:103140001EF00401630E826F3CEC0BF004012C0EA8
:10315000826F3CEC0BF066C100F167C101F168C100
:1031600002F169C103F101010A0E046F000E056F3F
:10317000000E066F000E076FE2EC1FF0000E046FEA
:10318000120E056F000E066F000E076F02EC20F0A6
:103190006FEC20F02AC182F40401300E82273CEC4F
:1031A0000BF02BC182F40401300E82273CEC0BF0B3
:1031B0002CC182F40401300E82273CEC0BF02DC1AF
:1031C00082F40401300E82273CEC0BF02EC182F415
:1031D0000401300E82273CEC0BF02FC182F4040175
:1031E000300E82273CEC0BF030C182F40401300E2B
:1031F00082273CEC0BF004012E0E826F3CEC0BF0AE
:1032000031C182F40401300E82273CEC0BF032C154
:1032100082F40401300E82273CEC0BF033C182F4BF
:103220000401300E82273CEC0BF00401730E826F18
:103230003CEC0BF004012C0E826F3CEC0BF0CCEC60
:1032400020F059C100F15AC101F142EC1BF095EC9C
:1032500012F013A27BEF19F004012C0E826F3CECEC
:103260000BF086C166F187C167F188C168F189C139
:1032700069F148EC14F00101000E046F000E056FB7
:10328000010E066F000E076F02EC20F06FEC20F0CD
:10329000296750EF19F00401200E826F53EF19F0E7
:1032A00004012D0E826F3CEC0BF030C182F404015E
:1032B000300E82273CEC0BF031C182F40401300E59
:1032C00082273CEC0BF004012E0E826F3CEC0BF0DD
:1032D00032C182F40401300E82273CEC0BF033C182
:1032E00082F40401300E82273CEC0BF004016D0ED9
:1032F000826F3CEC0BF013A4A2EF19F004012C0E2A
:10330000826F3CEC0BF013AC90EF19F00401500EFF
:10331000826F3CEC0BF0139C1398139AA2EF19F0F8
:1033200013AE9DEF19F00401460E826F3CEC0BF0DA
:10333000139E1398139AA2EF19F00401530E826F93
:103340003CEC0BF00FB2A8EF19F00FA0DAEF19F078
:1033500004012C0E826F3CEC0BF0200EF86EF76A25
:10336000F66A04010900F5CF82F43CEC0BF0090089
:10337000F5CF82F43CEC0BF00900F5CF82F43CEC85
:103380000BF00900F5CF82F43CEC0BF00900F5CF0F
:1033900082F43CEC0BF00900F5CF82F43CEC0BF02E
:1033A0000900F5CF82F43CEC0BF00900F5CF82F474
:1033B0003CEC0BF046EC0BF00F90109E129818EFBF
:1033C0001AF00401630E826F3CEC0BF004012C0E2A
:1033D000826F3CEC0BF01EEC1AF004012C0E826F95
:1033E0003CEC0BF091EC1AF004012C0E826F3CECDB
:1033F0000BF00DEC1BF004012C0E826F3CEC0BF07B
:103400000101F80E006FCD0E016F660E026F030E04
:10341000036F33EC1AF004012C0E826F3CEC0BF0BE
:1034200023EC1BF046EC0BF018EF1AF046EC0BF017
:103430000301C26B0790109227EF1DF0D8900E0E7B
:103440002DEC09F0E8CF00F10F0E2DEC09F0E8CFDC
:1034500001F1100E2DEC09F0E8CF02F1110E2DEC68
:1034600009F0E8CF03F10101000E046F000E056FB3
:10347000010E066F000E076F02EC20F06FEC20F0DB
:103480002AC182F40401300E82273CEC0BF02BC1E0
:1034900082F40401300E82273CEC0BF02CC182F444
:1034A0000401300E82273CEC0BF02DC182F40401A4
:1034B000300E82273CEC0BF02EC182F40401300E5A
:1034C00082273CEC0BF02FC182F40401300E8227DE
:1034D0003CEC0BF030C182F40401300E82273CEC4E
:1034E0000BF031C182F40401300E82273CEC0BF06A
:1034F00004012E0E826F3CEC0BF032C182F4040109
:10350000300E82273CEC0BF033C182F40401300E04
:1035100082273CEC0BF004016D0E826F3CEC0BF04B
:103520001200120E2DEC09F0E8CF00F1130E2DEC75
:1035300009F0E8CF01F1140E2DEC09F0E8CF02F10B
:10354000150E2DEC09F0E8CF03F101010A0E046F0E
:10355000000E056F000E066F000E076FE2EC1FF005
:10356000000E046F120E056F000E066F000E076F3F
:1035700002EC20F06FEC20F02AC182F40401300E3E
:1035800082273CEC0BF02BC182F40401300E822721
:103590003CEC0BF02CC182F40401300E82273CEC91
:1035A0000BF02DC182F40401300E82273CEC0BF0AD
:1035B0002EC182F40401300E82273CEC0BF02FC1A7
:1035C00082F40401300E82273CEC0BF030C182F40F
:1035D0000401300E82273CEC0BF004012E0E826FAA
:1035E0003CEC0BF031C182F40401300E82273CEC3C
:1035F0000BF032C182F40401300E82273CEC0BF058
:1036000033C182F40401300E82273CEC0BF004013C
:10361000730E826F3CEC0BF012000A0E2DEC09F0D9
:10362000E8CF00F10B0E2DEC09F0E8CF01F10C0E04
:103630002DEC09F0E8CF02F10D0E2DEC09F0E8CFEA
:1036400003F142EF1BF0060E2DEC09F0E8CF00F17C
:10365000070E2DEC09F0E8CF01F1080E2DEC09F072
:10366000E8CF02F1090E2DEC09F0E8CF03F142EFAB
:103670001BF00101CCEC20F0078457C100F158C1C8
:1036800001F107940101E80E046F800E056F000E32
:10369000066F000E076FE2EC1FF0000E046F040EC1
:1036A000056F000E066F000E076F02EC20F0880E0B
:1036B000046F130E056F000E066F000E076FD1EC3E
:1036C0001FF00A0E046F000E056F000E066F000E4D
:1036D000076F02EC20F06FEC20F00101296776EF14
:1036E0001BF00401200E826F79EF1BF004012D0EF8
:1036F000826F3CEC0BF030C182F40401300E822763
:103700003CEC0BF031C182F40401300E82273CEC1A
:103710000BF032C182F40401300E82273CEC0BF036
:1037200004012E0E826F3CEC0BF033C182F40401D5
:10373000300E82273CEC0BF00401430E826F3CEC10
:103740000BF0120087C32AF188C32BF189C32CF137
:103750008AC32DF18BC32EF18CC32FF18DC330F1B1
:103760008EC331F190C332F191C333F10101296B62
:103770001AEC21F091EC20F00101000E046F000E14
:10378000056F010E066F000E076FE2EC1FF00E0EC4
:103790000C6E00C10BF016EC09F00F0E0C6E01C19F
:1037A0000BF016EC09F0100E0C6E02C10BF016ECCB
:1037B00009F0110E0C6E03C10BF016EC09F00401B8
:1037C0007A0E826F3CEC0BF004012C0E826F3CEC05
:1037D0000BF00401350E826F3CEC0BF004012C0E53
:1037E000826F3CEC0BF01EEC1AF01EEF14F087C356
:1037F0002AF188C32BF189C32CF18AC32DF18BC325
:103800002EF18CC32FF18DC330F18EC331F190C3F3
:1038100032F191C333F10101296B1AEC21F091ECE3
:1038200020F0880E046F130E056F000E066F000E59
:10383000076FD6EC1FF0000E046F040E056F000E2C
:10384000066F000E076FE2EC1FF00101E80E046F37
:10385000800E056F000E066F000E076F02EC20F061
:103860000A0E0C6E00C10BF016EC09F00B0E0C6E7C
:1038700001C10BF016EC09F00C0E0C6E02C10BF03E
:1038800016EC09F00D0E0C6E03C10BF016EC09F0EE
:1038900004017A0E826F3CEC0BF004012C0E826F57
:1038A0003CEC0BF00401360E826F3CEC0BF0040193
:1038B0002C0E826F3CEC0BF00DEC1BF01EEF14F0A5
:1038C00087C32AF188C32BF189C32CF18AC32DF158
:1038D0008BC32EF18CC32FF18DC330F18FC331F127
:1038E00090C332F191C333F101011AEC21F091EC54
:1038F00020F0000E046F120E056F000E066F000E12
:10390000076FE2EC1FF001010A0E046F000E056F55
:10391000000E066F000E076F02EC20F0120E0C6E08
:1039200000C10BF016EC09F0130E0C6E01C10BF088
:1039300016EC09F0140E0C6E02C10BF016EC09F037
:10394000150E0C6E03C10BF016EC09F004017A0E93
:10395000826F3CEC0BF004012C0E826F3CEC0BF000
:103960000401370E826F3CEC0BF004012C0E826FC9
:103970003CEC0BF091EC1AF01EEF14F087C32AF127
:1039800088C32BF189C32CF18AC32DF18BC32EF18F
:103990008CC32FF18DC330F18EC331F190C332F15E
:1039A00091C333F10101296B1AEC21F091EC20F065
:1039B000880E046F130E056F000E066F000E076F62
:1039C000D6EC1FF0000E046F040E056F000E066F9C
:1039D000000E076FE2EC1FF00101E80E046F800E8D
:1039E000056F000E066F000E076F02EC20F0060E4A
:1039F0000C6E00C10BF016EC09F0070E0C6E01C145
:103A00000BF016EC09F0080E0C6E02C10BF016EC70
:103A100009F0090E0C6E03C10BF016EC09F004015D
:103A20007A0E826F3CEC0BF004012C0E826F3CECA2
:103A30000BF00401380E826F3CEC0BF004012C0EED
:103A4000826F3CEC0BF023EC1BF01EEF14F007A888
:103A50009AEF1DF00101800E006F1A0E016F060E25
:103A6000026F000E036F4BC104F14CC105F14DC153
:103A700006F14EC107F1D1EC1FF003BFE0EF1DF0DE
:103A80002CEC1EF04BC100F14CC101F14DC102F113
:103A90004EC103F10782DEEC1EF018C104F119C11A
:103AA00005F11AC106F11BC107F1F80E006FCD0E2A
:103AB000016F660E026F030E036FD1EC1FF00E0E46
:103AC0000C6E00C10BF016EC09F00F0E0C6E01C16C
:103AD0000BF016EC09F0100E0C6E02C10BF016EC98
:103AE00009F0110E0C6E03C10BF016EC09F00784FF
:103AF0000101CCEC20F057C100F158C101F107944D
:103B00000A0E0C6E00C10BF016EC09F00B0E0C6ED9
:103B100001C10BF016EC09F00C0E0C6E02C10BF09B
:103B200016EC09F00D0E0C6E03C10BF016EC09F04B
:103B3000E0EF1DF007AAE0EF1DF007840101CCECD7
:103B400020F057C100F158C101F10794060E0C6E28
:103B500000C10BF016EC09F0070E0C6E01C10BF062
:103B600016EC09F0080E0C6E02C10BF016EC09F011
:103B7000090E0C6E03C10BF016EC09F0078462C14C
:103B800000F163C101F164C102F165C103F1079461
:103B9000120E0C6E00C10BF016EC09F0130E0C6E39
:103BA00001C10BF016EC09F0140E0C6E02C10BF003
:103BB00016EC09F0150E0C6E03C10BF016EC09F0B3
:103BC0000798079A0401805181197F0B0DE09EA888
:103BD000FED714EE00F081517F0BE126E750812BD8
:103BE0000F01AD6EE2EF1DF08EEF0AF018C100F18B
:103BF00019C101F11AC102F11BC103F1000E046FDA
:103C0000000E056F010E066F000E076F02EC20F02C
:103C100029A121EF1EF02051D8B421EF1EF018C1C8
:103C200000F119C101F11AC102F11BC103F1000E2B
:103C3000046F000E056F0A0E066F000E076F02EC90
:103C400020F0120001010451001305510113065127
:103C500002130751031312000101186B196B1A6B41
:103C60001B6B12002AC182F40401300E82273CEC47
:103C70000BF02BC182F40401300E82273CEC0BF0D8
:103C80002CC182F40401300E82273CEC0BF02DC1D4
:103C900082F40401300E82273CEC0BF02EC182F43A
:103CA0000401300E82273CEC0BF02FC182F404019A
:103CB000300E82273CEC0BF030C182F40401300E50
:103CC00082273CEC0BF031C182F40401300E8227D4
:103CD0003CEC0BF032C182F40401300E82273CEC44
:103CE0000BF033C182F40401300E82273CEC0BF060
:103CF00012002FC182F40401300E82273CEC0BF03D
:103D000030C182F40401300E82273CEC0BF031C14B
:103D100082F40401300E82273CEC0BF032C182F4B5
:103D20000401300E82273CEC0BF033C182F4040115
:103D3000300E82273CEC0BF01200060E1E6E060EB3
:103D40001F6E060E206E1E2EA3EF1EF01F2EA3EF79
:103D50001EF0202EA3EF1EF08B84020E1E6E020EAC
:103D60001F6E020E206E1E2EB3EF1EF01F2EB3EF3D
:103D70001EF0202EB3EF1EF08B941200FF0E1F6E6C
:103D80001FC020F0030E1E6E8B841E2EC4EF1EF08B
:103D9000030E1E6E202EC4EF1EF08B941FC020F069
:103DA000030E1E6E1E2ED2EF1EF0030E1E6E203E60
:103DB000D2EF1EF01F2EC0EF1EF0120001010053C3
:103DC00005E1015303E1025301E1002BA1EC1FF0D7
:103DD000CCEC20F03951006F3A51016F420E046F64
:103DE0004B0E056F000E066F000E076FE2EC1FF022
:103DF00000C104F101C105F102C106F103C107F1DF
:103E000018C100F119C101F11AC102F11BC103F17E
:103E100007B20FEF1FF0D6EC1FF011EF1FF0D1EC3F
:103E20001FF000C118F101C119F102C11AF103C15B
:103E30001BF11200CCEC20F059C100F15AC101F184
:103E4000060E2DEC09F0E8CF04F1070E2DEC09F079
:103E5000E8CF05F1080E2DEC09F0E8CF06F1090EC8
:103E60002DEC09F0E8CF07F1D1EC1FF000C124F1EF
:103E700001C125F102C126F103C127F1290E046F0A
:103E8000000E056F000E066F000E076FE2EC1FF0CC
:103E9000EE0E046F430E056F000E066F000E076FE7
:103EA000D6EC1FF024C104F125C105F126C106F1AD
:103EB00027C107F1E2EC1FF000C11CF101C11DF1A7
:103EC00002C11EF103C11FF1120E2DEC09F0E8CF63
:103ED00004F1130E2DEC09F0E8CF05F1140E2DECD2
:103EE00009F0E8CF06F1150E2DEC09F0E8CF07F147
:103EF0000D0E006F000E016F000E026F000E036FBB
:103F0000E2EC1FF0180E046F000E056F000E066F36
:103F1000000E076F02EC20F01CC104F11DC105F179
:103F20001EC106F11FC107F1D6EC1FF06A0E046F27
:103F30002A0E056F000E066F000E076FD1EC1FF002
:103F40001200BF0EFA6E200E3A6F396BD890003710
:103F5000013702370337D8B0B2EF1FF03A2FA7EF7F
:103F60001FF039073A070353D8B412000331070B87
:103F700080093F6F03390F0B010F396F80EC5FF041
:103F8000406F390580EC5FF0405D405F396B3F3337
:103F9000D8B0392739333FA9C7EF1FF0405139272F
:103FA00012000101F1EC20F0D8B012000101035120
:103FB0000719346FB4EC20F0D8900751031934AFCF
:103FC000800F12000101346BD8EC20F0D8A0EEEC89
:103FD00020F0D8B01200C3EC20F0CCEC20F01F0E83
:103FE000366F04EC21F00B35D8B0B4EC20F0D8A03B
:103FF0000335D8B01200362FF1EF1FF034B1DBECEF
:1040000020F012000101346B045105110611071153
:104010000008D8A0D8EC20F0D8A0EEEC20F0D8B062
:104020001200086B096B0A6B0B6B04EC21F01F0E7E
:10403000366F04EC21F007510B5DD8A42CEF20F073
:1040400006510A5DD8A42CEF20F00551095DD8A4D3
:104050002CEF20F00451085DD8A03FEF20F0045170
:10406000085F0551D8A0053D095F0651D8A0063D5F
:104070000A5F0751D8A0073D0B5FD8900081362F0B
:1040800019EF20F034B1DBEC20F0346BD8EC20F0E9
:10409000D89008EC21F007510B5DD8A45CEF20F01C
:1040A00006510A5DD8A45CEF20F00551095DD8A443
:1040B0005CEF20F00451085DD8A06BEF20F0003FCA
:1040C0006BEF20F0013F6BEF20F0023F6BEF20F031
:1040D000032BD8B4120034B1DBEC20F01200010144
:1040E000346BD8EC20F0D8B012000DEC21F0200E8B
:1040F000366F003701370237033711EE33F00A0EFF
:10410000376FE7360A0EE75CD8B0E76EE552372F17
:1041100081EF20F0362F79EF20F034B12981D8904B
:10412000120001010A0E346F200E366F11EE29F0D5
:104130003451376F0A0ED890E652D8B0E726E732EE
:10414000372F9CEF20F00333023301330033362F37
:1041500096EF20F0E750FF0FD8A00335D8B012003B
:1041600029B1DBEC20F01200045100270551D8B032
:10417000053D01270651D8B0063D02270751D8B0AA
:10418000073D032712000051086F0151096F0251CA
:104190000A6F03510B6F12000101006B016B026B80
:1041A000036B12000101046B056B066B076B1200B9
:1041B0000335D8A012000351800B001F011F021FFE
:1041C000031F003FEBEF20F0013FEBEF20F0023F39
:1041D000EBEF20F0032B342B032512000735D8A07A
:1041E00012000751800B041F051F061F071F043F05
:1041F00001EF21F0053F01EF21F0063F01EF21F033
:10420000072B342B072512000037013702370337FD
:10421000083709370A370B3712000101296B2A6B5F
:104220002B6B2C6B2D6B2E6B2F6B306B316B326BC2
:10423000336B120001012A510F0B2A6F2B510F0B08
:104240002B6F2C510F0B2C6F2D510F0B2D6F2E51EF
:104250000F0B2E6F2F510F0B2F6F30510F0B306F35
:1042600031510F0B316F32510F0B326F33510F0B36
:04427000336F120096
:10BF0000E844F926000C160C2B0C3F0C520C640C68
:10BF1000760C860C960CA50CB30CC10CCF0CDC0C6B
:06BF2000E80CF40C000C1B
:00000001FF
